:020000040000FA
:040000000CEF12F0FF
:08000800FFEF0FF0D9CFE5FF77
:10001000E1CFD9FF00C0E5FF01C0E5FF02C0E5FF69
:1000200003C0E5FF04C0E5FF05C0E5FF06C0E5FF2E
:1000300007C0E5FF08C0E5FF09C0E5FF0AC0E5FF0E
:100040000BC0E5FF0CC0E5FF0DC0E5FF0EC0E5FFEE
:100050000FC0E5FF10C0E5FF11C0E5FF12C0E5FFCE
:1000600013C0E5FF14C0E5FF020EDBCF00F0030E66
:10007000DBCF01F0040EDBCF02F0050EDBCF03F087
:10008000060EDBCF04F0070EDBCF05F0080EDBCF4A
:1000900006F0090EDBCF07F00A0EDBCF08F00B0EDF
:1000A000DBCF09F00C0EDBCF0AF00D0EDBCF0BF02F
:1000B0000001C06B60AE29D0A49074AE13D009C00B
:1000C000E9FF0AC0F3FF0B50E0EC11F00C6E0C8658
:1000D0000CC0E5FF09C0E9FF0AC0F3FF0B5024EC98
:1000E00012F0749E0C6A60B00C2A0C50010BF46E76
:1000F0000001C051FE0BF4100001C06F0F0E0D6E19
:10010000600E0C6E800E0E6E40D00F0150AF3BD0D3
:10011000A49274AC13D009C0E9FF0AC0F3FF0B50DE
:10012000E0EC11F00F6E0F860FC0E5FF09C0E9FF8C
:100130000AC0F3FF0B5024EC12F0749C070E0F0161
:1001400050150F6E0F500001C06FC0C0E8FF020EC7
:100150000F5C12E209C0E9FF0AC0F3FF0B50E0ECAC
:1001600011F00F6E0F8E0FC0E5FF09C0E9FF0AC046
:10017000F3FF0B5024EC12F00F0E0D6E500E0C6EB0
:10018000800E0E6E02D0E86AFFD00CC00FF00DC0DA
:1001900010F00EC011F0000EE56E09C0E9FF0AC0B4
:1001A000F3FF0B5024EC12F00C50050F126E000EF2
:1001B0000D20136E000E0E20146E12C0E9FF13C046
:1001C000F3FF1450E0EC11F0126E12500001C16FF9
:1001D000C1C0E8FF0F0E121612C0E5FF06C0E9FF0E
:1001E00007C0F3FF085024EC12F00001C1AD12D09B
:1001F00009C0E9FF0AC0F3FF0B50E0EC11F0126EEA
:10020000128C12C0E5FF09C0E9FF0AC0F3FF0B50D2
:1002100024EC12F00C50020F126E000E0D20136E23
:10022000000E0E20146E12C0E9FF13C0F3FF14502D
:10023000E0EC11F0126E12500001C16F0001C1A775
:1002400016D009C0E9FF0AC0F3FF0B50E0EC11F033
:10025000126E128A12C0E5FF09C0E9FF0AC0F3FF5F
:100260000B5024EC12F0010E0001C16F02D000010E
:10027000C16B0C50010F126E000E0D20136E000E9C
:100280000E20146E0001C151E56E0250E56E015062
:10029000E56E0050E56E1450E56E1350E56E125099
:1002A000E56E4BEC05F0070EE126060E0C26000E5F
:1002B0000D22000E0E2206C0E9FF07C0F3FF085012
:1002C000E0EC11F0066E06500001C16F0CC000F0AA
:1002D0000DC001F00EC002F0066A06C007F0086A01
:1002E00006BE0868C1C00CF00D6A0850800FF36E9E
:1002F0000D50800FF35C02E10C50075C1DE200C062
:10030000E9FF01C0F3FF0250E0EC11F0076E002A94
:10031000D8B0012AD8B0022A07C0E5FF03C0E9FF20
:1003200004C0F3FF055024EC12F0032AD8B0042ACD
:10033000D8B0052A062AD1D7A4AE13D009C0E9FF48
:100340000AC0F3FF0B50E0EC11F0006E008800C013
:10035000E5FF09C0E9FF0AC0F3FF0B5024EC12F0DF
:10036000A49E0FC0E9FF10C0F3FF1150E0EC11F0A4
:10037000006E009E00C0E5FF0FC0E9FF10C0F3FF54
:10038000115024EC12F0010EE4CF14F0E4CF13F07E
:10039000E4CF12F0E4CF11F0E4CF10F0E4CF0FF08F
:1003A000E4CF0EF0E4CF0DF0E4CF0CF0E4CF0BF08F
:1003B000E4CF0AF0E4CF09F0E4CF08F0E4CF07F08F
:1003C000E4CF06F0E4CF05F0E4CF04F0E4CF03F08F
:1003D000E4CF02F0E4CF01F0E4CF00F0E4CFD9FFA6
:1003E0001200D9CFE5FFE1CFD9FF00C0E5FF01C082
:1003F000E5FF02C0E5FF03C0E5FF04C0E5FF05C05F
:10040000E5FF06C0E5FF07C0E5FF08C0E5FF09C03E
:10041000E5FF0AC0E5FF0BC0E5FF0CC0E5FF0DC01E
:10042000E5FF0EC0E5FF0FC0E5FF020EDBCF00F0D9
:10043000030EDBCF01F0040EDBCF02F0800EE56E81
:1004400089EC11F0E12A0F0E046E180E036E800E77
:10045000056E000EE56E000EE56E000EE56E070EF1
:10046000E56EFF0EE56E0550E56E0450E56E035037
:10047000E56EB3EC06F0080EE1260F0E046E1C0EBE
:10048000036E800E056E000EE56E000EE56E000E2A
:10049000E56E070EE56EFF0EE56E0550E56E045045
:1004A000E56E0350E56EB3EC06F0080EE126036A34
:1004B000046A056A066A0450800F800F02E1060E86
:1004C000035CD8B04BD105500024076E06500120C4
:1004D000086EE86A06BEE8680220096E07C0E9FFF8
:1004E00008C0F3FF0950A5EC11F0076EF3CF08F038
:1004F0000750FF0A04E10850FF0A01E12FD1830EE3
:100500000324096E000E04200A6E09C0E9FF0AC028
:10051000EAFFEFCF09F0060E095CD8B0F9D010C0A1
:10052000E5FF11C0E5FF116A09341136E8341136D0
:10053000FC0B106E000EFB6E050EFA6E540E1026AC
:100540001150FA22D8B0FB2A1050E4CF11F0E4CFBA
:1005500010F0F96EB6EF02F0D9EF02F0FCEF02F006
:100560001FEF03F042EF03F065EF03F00D01D481BC
:100570000F0E0A6E000E096E800E0B6E07C00CF097
:1005800008C00DF00E6A0F6A000EE56E0F50E56EA2
:100590000E50E56E0D50E56E0C50E56E0B50E56E9D
:1005A0000A50E56E0950E56EB3EC06F0080EE12640
:1005B000CDD00D01D4830F0E0A6E040E096E800E8D
:1005C0000B6E07C00CF008C00DF00E6A0F6A000E2B
:1005D000E56E0F50E56E0E50E56E0D50E56E0C5059
:1005E000E56E0B50E56E0A50E56E0950E56EB3EC12
:1005F00006F0080EE126AAD00D01D4850F0E0A6E72
:10060000080E096E800E0B6E07C00CF008C00DF0CE
:100610000E6A0F6A000EE56E0F50E56E0E50E56E25
:100620000D50E56E0C50E56E0B50E56E0A50E56E10
:100630000950E56EB3EC06F0080EE12687D00D01F7
:10064000D4870F0E0A6E0C0E096E800E0B6E07C05B
:100650000CF008C00DF00E6A0F6A000EE56E0F5028
:10066000E56E0E50E56E0D50E56E0C50E56E0B50CC
:10067000E56E0A50E56E0950E56EB3EC06F0080E23
:10068000E12664D00D01D4890F0E0A6E100E096E9A
:10069000800E0B6E07C00CF008C00DF00E6A0F6ADA
:1006A000000EE56E0F50E56E0E50E56E0D50E56ED6
:1006B0000C50E56E0B50E56E0A50E56E0950E56E84
:1006C000B3EC06F0080EE12641D00D01D48B0F0EDD
:1006D0000A6E140E096E800E0B6E07C00CF008C077
:1006E0000DF00E6A0F6A000EE56E0F50E56E0E50AB
:1006F000E56E0D50E56E0C50E56E0B50E56E0A5040
:10070000E56E0950E56EB3EC06F0080EE1261ED04A
:100710000D01D48B0F0E0A6E140E096E800E0B6E37
:100720000C6A0D6A000EE56E0D50E56E0C50E56E1C
:100730000850E56E0750E56E0B50E56E0A50E56E09
:100740000950E56EB3EC06F0080EE126020E052610
:10075000D8B0062A032AD8B0042AADD6000EE56E1A
:1007600089EC11F0E12AF36AE86AE4CF0FF0E4CFF4
:100770000EF0E4CF0DF0E4CF0CF0E4CF0BF0E4CFBB
:100780000AF0E4CF09F0E4CF08F0E4CF07F0E4CFBB
:1007900006F0E4CF05F0E4CF04F0E4CF03F0E4CFBB
:1007A00002F0E4CF01F0E4CF00F0E4CFD9FF120073
:1007B000D9CFE5FFE1CFD9FF00C0E5FF01C0E5FFDC
:1007C00002C0E5FF03C0E5FF04C0E5FF05C0E5FF8B
:1007D00006C0E5FF07C0E5FF08C0E5FF09C0E5FF6B
:1007E0000AC0E5FF0BC0E5FF0CC0E5FF0DC0E5FF4B
:1007F0000EC0E5FF0FC0E5FF10C0E5FF11C0E5FF2B
:1008000012C0E5FF13C0E5FF14C0E5FF15C0E5FF0A
:10081000020EDBCF00F0030EDBCF01F0040EDBCFC6
:1008200002F0050EDBCF03F0060EDBCF04F0070E5F
:10083000DBCF05F0080EDBCF06F0090EDBCF07F0AB
:100840000A0EDBCF08F00F0E0A6E400E096E800E06
:100850000B6E09500001606F0A500001616F0B5070
:100860000001626F0F0E0A6E300E096E800E0B6E65
:1008700009500001636F0A500001646F0B500001C2
:10088000656F0F0E0A6E200E096E800E0B6E0950FA
:100890000001666F0A500001676F0B500001686F1E
:1008A000096A0A6A020E095CD8B0C5D0600E0A2433
:1008B0000B6E0C6A000E0C220BC0E9FF0CC0EAFFA5
:1008C000EECF0BF0EECF0CF0EFCF0DF00BC00EF033
:1008D0000CC00FF00DC010F00BC0E9FF0CC0F3FF0F
:1008E0000D50E0EC11F0116E11B6A1D0FC0E1116F6
:1008F00011C0E5FF0BC0E9FF0CC0F3FF0D5024EC65
:1009000012F00BC0E9FF0CC0F3FF0D50E0EC11F04A
:10091000116E030E0814126E1250111211C0E5FF71
:100920000BC0E9FF0CC0F3FF0D5024EC12F008AC33
:1009300004D0400E0710116E02D007C011F00B500A
:10094000050F126E000E0C20136E000E0D20146E9B
:1009500011C0E5FF12C0E9FF13C0F3FF145024ECEF
:1009600012F008AA03D0010E116E01D0116A0B50CB
:10097000010F126E000E0C20136E000E0D20146E6F
:100980001150E56E0350E56E0250E56E0150E56EC4
:100990000050E56E1450E56E1350E56E1250E56E92
:1009A000B3EC06F0080EE126060E0B26000E0C2214
:1009B000000E0D2204C011F005C012F006C013F0A5
:1009C000146A0750145C1DE211C0E9FF12C0F3FF66
:1009D0001350E0EC11F0156E112AD8B0122AD8B0DD
:1009E000132A15C0E5FF0BC0E9FF0CC0F3FF0D5043
:1009F00024EC12F00B2AD8B00C2AD8B00D2A142AF5
:100A0000E0D70EC0E9FF0FC0F3FF1050E0EC11F08B
:100A10000B6E0BB40AD00B860BC0E5FF0EC0E9FFCE
:100A20000FC0F3FF105024EC12F0010E05D0030E9E
:100A30000A26092A37D7E86AE4CF15F0E4CF14F084
:100A4000E4CF13F0E4CF12F0E4CF11F0E4CF10F0D4
:100A5000E4CF0FF0E4CF0EF0E4CF0DF0E4CF0CF0D4
:100A6000E4CF0BF0E4CF0AF0E4CF09F0E4CF08F0D4
:100A7000E4CF07F0E4CF06F0E4CF05F0E4CF04F0D4
:100A8000E4CF03F0E4CF02F0E4CF01F0E4CF00F0D4
:100A9000E4CFD9FF1200D9CFE5FFE1CFD9FF00C0E5
:100AA000E5FF01C0E5FF02C0E5FF03C0E5FF04C0AC
:100AB000E5FF05C0E5FF06C0E5FF07C0E5FF08C08C
:100AC000E5FF09C0E5FF0AC0E5FF0BC0E5FF0CC06C
:100AD000E5FF0DC0E5FF020EDBCF00F0030EDBCF1C
:100AE00001F0040EDBCF02F0050EDBCF03F0060EA3
:100AF000DBCF04F0070EDBCF05F0080EDBCF06F0EE
:100B00000650D8A46CD000C0E9FF01C0F3FF02502A
:100B1000E0EC11F0066E0638E840F80B076E07C0EF
:100B2000E5FF03C0E9FF04C0F3FF055024EC12F019
:100B30000350010F086E000E0420096E000E052000
:100B40000A6E0638E840070B066E06C0E5FF08C0CF
:100B5000E9FF09C0F3FF0A5024EC12F0002AD8B0D4
:100B6000012AD8B0022A00C0E9FF01C0F3FF0250F9
:100B7000E0EC11F0066E0638E840070B066E0650F2
:100B8000071207C0E5FF03C0E9FF04C0F3FF0550EB
:100B900024EC12F00350020F066E000E0420076EC4
:100BA000000E0520086E000EE56E06C0E9FF07C0C6
:100BB000F3FF085024EC12F00350030F066E000EF2
:100BC0000420076E000E0520086E000EE56E06C0BC
:100BD000E9FF07C0F3FF085024EC12F0A5D0035042
:100BE000020F066E000E0420076E000E0520086E30
:100BF00000C0E9FF01C0F3FF0250E0EC11F0096E04
:100C00000938E844E00B0A6E0AC0E5FF06C0E9FFB8
:100C100007C0F3FF085024EC12F00350030F0B6ED3
:100C2000000E04200C6E000E05200D6E0938E844FD
:100C30001F0B096E09C0E5FF0BC0E9FF0CC0F3FFF5
:100C40000D5024EC12F0002AD8B0012AD8B0022AA4
:100C500006C0E9FF07C0F3FF0850E0EC11F0E86EB2
:100C600000C0E9FF01C0F3FF0250E0EC11F0096E93
:100C7000030E09140B6E0B500A120AC0E5FF06C0E2
:100C8000E9FF07C0F3FF085024EC12F006C0E9FFAB
:100C900007C0F3FF0850E0EC11F0E86EE00E091613
:100CA0000938E8441F0B096E09500A120AC0E5FF13
:100CB00006C0E9FF07C0F3FF085024EC12F0002A39
:100CC000D8B0012AD8B0022A0350010F066E000ED8
:100CD0000420076E000E0520086E00C0E9FF01C069
:100CE000F3FF0250E0EC11F0096E09C0E5FF06C009
:100CF000E9FF07C0F3FF085024EC12F0002AD8B037
:100D0000012AD8B0022A00C0E9FF01C0F3FF025057
:100D1000E0EC11F0006E00C0E5FF03C0E9FF04C085
:100D2000F3FF055024EC12F0E4CF0DF0E4CF0CF00B
:100D3000E4CF0BF0E4CF0AF0E4CF09F0E4CF08F001
:100D4000E4CF07F0E4CF06F0E4CF05F0E4CF04F001
:100D5000E4CF03F0E4CF02F0E4CF01F0E4CF00F001
:100D6000E4CFD9FF1200D9CFE5FFE1CFD9FF00C012
:100D7000E5FF01C0E5FF02C0E5FF03C0E5FF04C0D9
:100D8000E5FF05C0E5FF06C0E5FF07C0E5FF08C0B9
:100D9000E5FF09C0E5FF0AC0E5FF020EDBCF00F06A
:100DA000030EDBCF01F0040EDBCF02F0050EDBCF2C
:100DB000B3F0060EDBCFB4F0070EDBCFB5F0080EB4
:100DC000DBCFB6F0090EDBCF03F0000E056EB30EDD
:100DD000046E800E066E0350D8A450D004C0E9FF04
:100DE00005C0F3FF0650E0EC11F0036E0338E84451
:100DF0001F0B076E07C0E5FF00C0E9FF01C0F3FF4E
:100E0000025024EC12F000C0E9FF01C0F3FF0250D1
:100E1000E0EC11F0076E0450010F086E000E052083
:100E2000096E000E06200A6E08C0E9FF09C0F3FF34
:100E30000A50E0EC11F0086E0838E844E00B096E47
:100E40000950071207C0E5FF00C0E9FF01C0F3FF2A
:100E5000025024EC12F0002AD8B0012AD8B0022A9D
:100E60000338E844E00B076E07C0E5FF00C0E9FF68
:100E700001C0F3FF025024EC12F0A6D00450020F80
:100E8000036E000E0520076E000E0620086E03C0DC
:100E9000E9FF07C0F3FF0850E0EC11F0036E0338E0
:100EA000E840070B076E07C0E5FF00C0E9FF01C07F
:100EB000F3FF025024EC12F000C0E9FF01C0F3FF81
:100EC0000250E0EC11F0076E0450030F086E000EA4
:100ED0000520096E000E06200A6E08C0E9FF09C051
:100EE000F3FF0A50E0EC11F0086E0838E840F80B08
:100EF000096E0950071207C0E5FF00C0E9FF01C0F5
:100F0000F3FF025024EC12F0002AD8B0012AD8B026
:100F1000022A0338E840F80B076EE00E071607C0F8
:100F2000E5FF00C0E9FF01C0F3FF025024EC12F01E
:100F3000078607C0E5FF00C0E9FF01C0F3FF0250CC
:100F400024EC12F0030E03160350071207C0E5FF4E
:100F500000C0E9FF01C0F3FF025024EC12F0002AA8
:100F6000D8B0012AD8B0022A0450010F036E000E37
:100F70000520076E000E0620086E03C0E9FF07C0BB
:100F8000F3FF0850E0EC11F0036E03C0E5FF00C072
:100F9000E9FF01C0F3FF025024EC12F0002AD8B0A0
:100FA000012AD8B0022A04C0E9FF05C0F3FF0650A9
:100FB000E0EC11F0046E04C0E5FF00C0E9FF01C0E1
:100FC000F3FF025024EC12F0E4CF0AF0E4CF09F072
:100FD000E4CF08F0E4CF07F0E4CF06F0E4CF05F06B
:100FE000E4CF04F0E4CF03F0E4CF02F0E4CF01F06B
:100FF000E4CF00F0E4CFD9FF1200D9CFE5FFE1CF75
:10100000D9FF00C0E5FF01C0E5FF02C0E5FF03C056
:10101000E5FF04C0E5FF05C0E5FF06C0E5FF07C02A
:10102000E5FF08C0E5FF09C0E5FF020EDBCF00F0D9
:10103000030EDBCF01F0040EDBCF02F0050EDBCF99
:1010400003F0060EDBCF04F00050010A02E101506C
:1010500001E0EAD002C0E9FF03C0F3FF0450A5ECB1
:1010600011F0006EF3CF01F00150E56E0050E56E17
:10107000000EE56E020EE56E4BEC0EF0026EF3CF45
:1010800003F0040EE126046A056A400E02264B0EA8
:1010900003224C0E0422000E052200C006F001C0FF
:1010A00007F0086A096A0950E56E0850E56E0750B6
:1010B000E56E0650E56E0550E56E0450E56E035092
:1010C000E56E0250E56E10EC0AF0026EF3CF03F00D
:1010D000F4CF04F0E9CF05F0080EE126000EE56E2E
:1010E000000EE56E000EE56E040EE56E0550E56E31
:1010F0000450E56E0350E56E0250E56E10EC0AF008
:10110000026EF3CF03F0F4CF04F0E9CF05F0080E40
:10111000E126FF0E0226FF0E0322FF0E0422FF0E21
:1011200005220550800F800F08E1000E045C05E1E8
:10113000010E035C02E1000E025C0AE20350E56E60
:101140000250E56E7C0EC0EC0FF0020EE12664D07A
:101150000150E56E0050E56E000EE56E080EE56E7E
:101160004BEC0EF0006EF3CF01F0040EE126046AA2
:10117000056A400E00264B0E01224C0E0422000E82
:1011800005220950E56E0850E56E0750E56E0650E1
:10119000E56E0550E56E0450E56E0150E56E0050B9
:1011A000E56E10EC0AF0006EF3CF01F0F4CF04F01E
:1011B000E9CF05F0080EE126000EE56E000EE56EA3
:1011C000000EE56E100EE56E0550E56E0450E56EFE
:1011D0000150E56E0050E56E10EC0AF0006EF3CFA2
:1011E00001F0F4CF04F0E9CF05F0080EE126FF0E80
:1011F0000026FF0E0122FF0E0422FF0E05220050E2
:10120000026E0150036E0350E56E0250E56E6C0EE7
:10121000C0EC0FF0020EE1260D0E36EC12F0AB8E94
:10122000AB88F36A010E02D0F36AE86AE4CF09F0F2
:10123000E4CF08F0E4CF07F0E4CF06F0E4CF05F008
:10124000E4CF04F0E4CF03F0E4CF02F0E4CF01F008
:10125000E4CF00F0E4CFD9FF1200006A016A000178
:10126000B76B060E0001B86F770E00018A6F010E92
:1012700000018B6F040E00018C6F010E00018D6F59
:1012800000018E6B040E00018F6F030E0001906F42
:101290000001A46BE10E0001A56F010E0001A76F14
:1012A000000E036EA40E026E800E046E0450E56EF6
:1012B0000350E56E0250E56E000EE56E010EE56E20
:1012C000FDEC07F0050EE126000E036EB70E026E70
:1012D000800E046E0450E56E0350E56E0250E56E1C
:1012E000000EE56E47EC0DF0040EE1266EEC10F0FA
:1012F000FFEC11F093928A92AA0EE56E000EE56E55
:10130000010EE56ED6EC10F0030EE126002AD8B0EF
:10131000012A00504C0A03E101501D0A01E007D0E8
:10132000000EE56EA2EC10F0E12A006A016A000EE0
:10133000036E970E026E800E046E0450E56E03502D
:10134000E56E0250E56EE7EC0AF0026EF3CF03F0B3
:10135000030EE1260350800F800F02E1010E025CB4
:1013600036E300019951E56E000EE56E010EE56E63
:10137000D6EC10F0030EE12600019751026E0250E8
:10138000E56E000EE56E010EE56ED6EC10F0030E74
:10139000E12600019851026E036A0250E56E000ECC
:1013A000E56E010EE56ED6EC10F0030EE126000EA0
:1013B000036E8A0E026E800E046E0450E56E0350BA
:1013C000E56E0250E56E42EC0CF0030EE126015092
:1013D000800F460F02E1990E005C02E38A8201D081
:1013E0008A92000EE56E010EE56E69EC11F0026E58
:1013F000020EE1260250D8B489D7000EE56E010E28
:10140000E56E47EC11F0026E020EE1260250E56E29
:10141000000EE56E37EC10F0020EE12677D71200D1
:10142000D9CFE5FFE1CFD9FF00C0E5FF01C0E5FF5F
:1014300002C0E5FF03C0E5FF04C0E5FF05C0E5FF0E
:1014400006C0E5FF07C0E5FF08C0E5FF09C0E5FFEE
:101450000AC0E5FF0BC0E5FF0CC0E5FF0DC0E5FFCE
:10146000020EDBCF00F0030EDBCF01F0040EDBCF6A
:1014700002F0050EDBCF03F0060EDBCF04F0070E03
:10148000DBCF05F0080EDBCF06F0090EDBCF07F04F
:10149000D88003AED890086A083608500FE0031CC5
:1014A0000C6E021C0B6E011C0A6E001C096E092AD0
:1014B0000DE10A2A0BE10B4A0C2A08D000C009F002
:1014C00001C00AF002C00BF003C00CF009C000F02C
:1014D0000AC001F00BC002F00CC003F0D88007AEC8
:1014E000D890096A093609500FE0071C0D6E061CDA
:1014F0000C6E051C0B6E041C0A6E0A2A0DE10B2AE9
:101500000BE10C4A0D2A08D004C00AF005C00BF00C
:1015100006C00CF007C00DF00D50E56E0C50E56EE6
:101520000B50E56E0A50E56E0350E56E0250E56E15
:101530000150E56E0050E56EB5EC0BF0006EF3CF98
:1015400001F0F4CF02F0E9CF03F0080EE1260950D4
:10155000081A085016E0031C076E021C066E011CD8
:10156000056E001C046E042A04E1052A02E1064A05
:10157000072A07C0E9FF06C0F4FF05C0F3FF0450C7
:1015800007D003C0E9FF02C0F4FF01C0F3FF005021
:10159000E4CF0DF0E4CF0CF0E4CF0BF0E4CF0AF091
:1015A000E4CF09F0E4CF08F0E4CF07F0E4CF06F091
:1015B000E4CF05F0E4CF04F0E4CF03F0E4CF02F091
:1015C000E4CF01F0E4CF00F0E4CFD9FF1200D9CF8F
:1015D000E5FFE1CFD9FF00C0E5FF01C0E5FF02C094
:1015E000E5FF03C0E5FF04C0E5FF05C0E5FF06C059
:1015F000E5FF07C0E5FF08C0E5FF09C0E5FF0AC039
:10160000E5FF0BC0E5FF0CC0E5FF0DC0E5FF0EC018
:10161000E5FF020EDBCF00F0030EDBCF01F0040E7E
:10162000DBCF02F0000E046EAF0E036E800E056E6F
:101630000050030F066E000E0120076E000E022000
:10164000086E0050020F096E000E01200A6E000E97
:1016500002200B6E000E0D6EBF0E0C6E800E0E6E15
:101660000E50E56E0D50E56E0C50E56E0B50E56EBC
:101670000A50E56E0950E56E0850E56E0750E56EBC
:101680000650E56E0550E56E0450E56E0350E56EBC
:1016900006EC00F0036E0C0EE126035003E1F36A42
:1016A000E86A42D00001AF51036E0001B051046EF0
:1016B00003C0E5FF04C0F4FF00C0E9FF01C0F3FF71
:1016C000025018EC12F0ACC003F0032A03500001E2
:1016D000AC6F0001BF51600B09E0AEC003F0032AFC
:1016E00003500001AE6FF368E8681ED00001BFA789
:1016F00009D0ADC003F0032A03500001AD6FF368B9
:10170000FE0E12D0020E0026000E0122000E022252
:1017100000C0E9FF01C0F3FF0250E0EC11F0006EE1
:10172000016A01C0F3FF0050E4CF0EF0E4CF0DF0EA
:10173000E4CF0CF0E4CF0BF0E4CF0AF0E4CF09F0F3
:10174000E4CF08F0E4CF07F0E4CF06F0E4CF05F0F3
:10175000E4CF04F0E4CF03F0E4CF02F0E4CF01F0F3
:10176000E4CF00F0E4CFD9FF1200D9CFE5FFE1CFFD
:10177000D9FF00C0E5FF01C0E5FF02C0E5FF03C0DF
:10178000E5FF04C0E5FF05C0E5FF06C0E5FF07C0B3
:10179000E5FF08C0E5FF09C0E5FF0AC0E5FF0BC093
:1017A000E5FF0CC0E5FF0DC0E5FF020EDBCF00F04A
:1017B000030EDBCF01F0040EDBCF02F0050EDBCF12
:1017C00003F0060EDBCF04F0070EDBCF05F0080EAA
:1017D000DBCF06F0090EDBCF07F0086A096A0A6A58
:1017E0000B6A200E0C6E0344010B0D6E010E0D16DC
:1017F0000050002601360236033608500826093606
:101800000A360B360D50D8A4088007500B5C08E14F
:1018100006500A5C05E10550095C02E10450085CD1
:1018200009E30450085E0550095A06500A5A075049
:101830000B5A00800C2ED7D703C0E9FF02C0F4FF7B
:1018400001C0F3FF0050E4CF0DF0E4CF0CF0E4CF83
:101850000BF0E4CF0AF0E4CF09F0E4CF08F0E4CFD6
:1018600007F0E4CF06F0E4CF05F0E4CF04F0E4CFD6
:1018700003F0E4CF02F0E4CF01F0E4CF00F0E4CFD6
:10188000D9FF1200D9CFE5FFE1CFD9FF00C0E5FFB6
:1018900001C0E5FF02C0E5FF03C0E5FF04C0E5FFAE
:1018A00005C0E5FF06C0E5FF07C0E5FF08C0E5FF8E
:1018B00009C0E5FF020EDBCF00F0030EDBCF01F025
:1018C000040EDBCF02F000C0E9FF01C0F3FF0250BD
:1018D000A5EC11F0036EF3CF04F0056A066A005020
:1018E000030F076E000E0120086E000E0220096E25
:1018F000020E0026000E0122000E022200C0E9FFA7
:1019000001C0F3FF0250E0EC11F0006E000EE56E36
:101910000050E56E0950E56E0850E56E0750E56E23
:101920000650E56E0550E56E0450E56E0350E56E19
:10193000D8EC03F0006E090EE126016A0050011098
:1019400007E0AAC002F0022A02500001AA6F06D0E6
:10195000ABC002F0022A02500001AB6F01C0F3FFDE
:101960000050E4CF09F0E4CF08F0E4CF07F0E4CF73
:1019700006F0E4CF05F0E4CF04F0E4CF03F0E4CFC9
:1019800002F0E4CF01F0E4CF00F0E4CFD9FF120081
:10199000D9CFE5FFE1CFD9FF00C0E5FF01C0E5FFEA
:1019A00002C0E5FF03C0E5FF04C0E5FF05C0E5FF99
:1019B00006C0E5FF07C0E5FF08C0E5FF09C0E5FF79
:1019C0000AC0E5FF0BC0E5FF020EDBCF00F0030EFF
:1019D000DBCF01F0040EDBCF02F0050EDBCF03F00E
:1019E000060EDBCF04F0070EDBCF05F0080EDBCFD1
:1019F00006F00050010A02E1015001E02DD0076A13
:101A0000086A0850800FF36E0650800FF35C02E105
:101A10000550075C21E207500224096E085003209C
:101A20000A6EE86A08BEE86804200B6E09C0E9FF88
:101A30000AC0F3FF0B50E0EC11F0096E0950E56E9F
:101A40000150E56E0050E56ED6EC10F0030EE12675
:101A5000072AD8B0082AD5D7E4CF0BF0E4CF0AF094
:101A6000E4CF09F0E4CF08F0E4CF07F0E4CF06F0CC
:101A7000E4CF05F0E4CF04F0E4CF03F0E4CF02F0CC
:101A8000E4CF01F0E4CF00F0E4CFD9FF1200D9CFCA
:101A9000E5FFE1CFD9FF00C0E5FF01C0E5FF02C0CF
:101AA000E5FF03C0E5FF020EDBCF00F0030EDBCF46
:101AB00001F0040EDBCF02F0050EDBCF03F0030EC6
:101AC000005CD8B03CD004C0E5FF05C0E5FF056A66
:101AD00000340536E8340536FC0B046E000EFB6E50
:101AE0001A0EFA6EFC0E04260550FA22D8B0FB2A14
:101AF0000450E4CF05F0E4CF04F0F96E84EF0DF06C
:101B00009FEF0DF09FEF0DF0012AD8B0022AD8B058
:101B1000032A01C0E9FF02C0F3FF0350E0EC11F01B
:101B2000006E080E005C09E2D56A800ED510016EC9
:101B300000500110D56E010E03D0E86A01D0E86AAA
:101B4000E4CF03F0E4CF02F0E4CF01F0E4CF00F003
:101B5000E4CFD9FF1200D9CFE5FFE1CFD9FF00C014
:101B6000E5FF01C0E5FF02C0E5FF03C0E5FF04C0DB
:101B7000E5FF05C0E5FF06C0E5FF07C0E5FF020E73
:101B8000DBCF00F0030EDBCF01F0040EDBCF02F061
:101B9000050EDBCF03F0060EDBCF04F0056A045020
:101BA000055C15E205500024066E01C0E9FF02C085
:101BB000F3FF0350E0EC11F0076E0750E56E06509E
:101BC000E56E37EC10F0020EE126052AE8D7045046
:101BD000E4CF07F0E4CF06F0E4CF05F0E4CF04F063
:101BE000E4CF03F0E4CF02F0E4CF01F0E4CF00F063
:101BF000E4CFD9FF1200D9CFE5FFE1CFD9FF00C074
:101C0000E5FF01C0E5FF02C0E5FF03C0E5FF04C03A
:101C1000E5FF05C0E5FF06C0E5FF07C0E5FF020ED2
:101C2000DBCF00F0030EDBCF01F0040EDBCF02F0C0
:101C3000050EDBCF03F0060EDBCF04F0056A04507F
:101C4000055C15E205500024066E01C0E9FF02C0E4
:101C5000F3FF0350E0EC11F0076E0750E56E0650FD
:101C6000E56E37EC10F0020EE126052AE8D70450A5
:101C7000E4CF07F0E4CF06F0E4CF05F0E4CF04F0C2
:101C8000E4CF03F0E4CF02F0E4CF01F0E4CF00F0C2
:101C9000E4CFD9FF1200D9CFE5FFE1CFD9FF00C0D3
:101CA000E5FF01C0E5FF02C0E5FF03C0E5FF020E4E
:101CB000DBCF00F0030EDBCF01F0040EDBCF02F030
:101CC000050EDBCF03F000500001B96F0150BA6F71
:101CD00002500001BB6F0350BC6F0001B9510001FD
:101CE000BB03F3CF00F0F4CF01F000500001BD6F53
:101CF0000150BE6F0001B9510001BC03F3CF00F0E9
:101D00000001BA510001BB03F3CF01F001500026DE
:101D10000001BE5100260050BE6FBEC0F3FFBD5192
:101D2000E4CF03F0E4CF02F0E4CF01F0E4CF00F021
:101D3000E4CFD9FF1200B40EF66E240EF76E000E3B
:101D4000F86E0900F550056E0900F550066E055055
:101D500002E106503BE00900F550006E0900F55025
:101D6000016E0900F550026E09000900F550E96E98
:101D70000900F550EA6E090009000900F550036EEC
:101D80000900F550046E09000900F6CF07F0F7CFFF
:101D900008F0F8CF09F000C0F6FF01C0F7FF02C05D
:101DA000F8FF035002E1045007E00900F550EE6E21
:101DB0000306F8E20406F9D707C0F6FF08C0F7FFEC
:101DC00009C0F8FF0506C4E20606C5D71200D9CF40
:101DD000E5FFE1CFD9FF00C0E5FF01C0E5FF02C08C
:101DE000E5FF03C0E5FF04C0E5FF05C0E5FF06C051
:101DF000E5FF020EDBCF00F0030EDBCF01F0040E97
:101E0000DBCF02F0050EDBCF03F0060EDBCF04F0D4
:101E1000056A0450055C14E205500324066E065062
:101E2000E56EF1EC11F0066EE12A06C0E5FF00C098
:101E3000E9FF01C0F3FF025024EC12F0052AE9D7B4
:101E40000450E4CF06F0E4CF05F0E4CF04F0E4CF93
:101E500003F0E4CF02F0E4CF01F0E4CF00F0E4CFF0
:101E6000D9FF1200D9CFE5FFE1CFD9FF00C0E5FFD0
:101E700001C0E5FF02C0E5FF03C0E5FF04C0E5FFC8
:101E800005C0E5FF06C0E5FF020EDBCF00F0030E44
:101E9000DBCF01F0040EDBCF02F0050EDBCF03F049
:101EA000060EDBCF04F0056A0450055C14E2055011
:101EB0000324066E0650E56EF1EC11F0066EE12A81
:101EC00006C0E5FF00C0E9FF01C0F3FF025024ECAB
:101ED00012F0052AE9D70450E4CF06F0E4CF05F06C
:101EE000E4CF04F0E4CF03F0E4CF02F0E4CF01F05C
:101EF000E4CF00F0E4CFD9FF1200D9CFE5FFE1CF66
:101F0000D9FF800EE56E89EC11F0E12A010E706EAA
:101F1000AE0E716E050E726E200E736E779E779CFC
:101F2000040E606E0F01506B0F01006B0F01016B0F
:101F30000F01046B0F01056B0F01086B0F01096B9B
:101F40000F010C6B0F010D6B0F01106B0F01116B6B
:101F50000F01146B0F01156B0F01186B0F01196B3B
:101F60000F0119970F011C6B0F011D6B0F011D97BE
:101F7000000EE56E89EC11F0E12AE4CFD9FF1200E2
:101F8000D9CFE5FFE1CFD9FF00C0E5FF01C0E5FFF4
:101F900002C0E5FF006E020EDBCF01F0030EDBCFC7
:101FA00002F0AC6AAB6A00B0AC8800A202D0AC8C84
:101FB000AB8C00A401D0AC8E00A602D0AB8801D0BF
:101FC000AB8A00A802D0AC8401D0AC949E9800AC3F
:101FD00002D09D8A01D09D9A9E9A00AE02D09D8823
:101FE00001D09D980150AF6EAC8AAB8EE4CF02F069
:101FF000E4CF01F0E4CF00F0E4CFD9FF1200E8CF46
:10200000E5FFD8CFE5FFE0CFE5FFF3CFE5FFF4CF65
:10201000E5FFE9CFE5FFEACFE5FFFACFE5FFFBCF2C
:10202000E5FFD9CFE5FFE1CFD9FF00C0E5FF006AAA
:10203000F2B4002A0050010A03E1CFEC11F0F2944F
:10204000E4CF00F0E4CFD9FFE4CFFBFFE4CFFAFF09
:10205000E4CFEAFFE4CFE9FFE4CFF4FFE4CFF3FFFE
:10206000E4CFE0FFE4CFD8FFE4CFE8FF1000D9CF02
:10207000E5FFE1CFD9FF00C0E5FF020EDBCF00F0A6
:10208000030EDBCFA8FF00C0A9FFA69EA69CA684D6
:10209000F29E550EA76EAA0EA76EA682A6A202D029
:1020A0000000FCD7A6A613D0450E36EC12F061EC6A
:1020B00012F0006E0050FBE1520E36EC12F061ECB3
:1020C00012F0006E0050FBE1520E36EC12F0A694B6
:1020D000F28EE4CF00F0E4CFD9FF1200D9CFE5FFB4
:1020E000E1CFD9FF00C0E5FF01C0E5FF02C0E5FF79
:1020F00003C0E5FF7DEC0FF0006A016A0150800F1C
:10210000800F02E1050E005C10E2AA0E0024026EB0
:10211000000E0120036E02C0E9FF03C0EAFF000EBB
:10212000EF6E002AD8B0012AE9D7F36AE86AE4CF53
:1021300003F0E4CF02F0E4CF01F0E4CF00F0E4CF0D
:10214000D9FF1200D9CFE5FFE1CFD9FF00C0E5FFED
:1021500001C0E5FF02C0E5FF03C0E5FF04C0E5FFE5
:1021600005C0E5FF020EDBCF00F0005010E1D6CF36
:1021700000F0016AD7CF02F0036A0250056E046ACC
:10218000045000260550012201C0F3FF0050E4CFA7
:1021900005F0E4CF04F0E4CF03F0E4CF02F0E4CFA5
:1021A00001F0E4CF00F0E4CFD9FF1200D9CFE5FF72
:1021B000E1CFD9FF00C0E5FF01C0E5FF02C0E5FFA8
:1021C000020EDBCF00F0030EDBCF01F0040EDBCFFD
:1021D00002F00050010A02E1015001E008D0025073
:1021E00036EC12F061EC12F0006E0050FBE1E4CF2F
:1021F00002F0E4CF01F0E4CF00F0E4CFD9FF120009
:10220000D9CFE5FFE1CFD9FF00C0E5FF01C0E5FF71
:1022100002C0E5FF03C0E5FF020EDBCF00F0030EB6
:10222000DBCF01F00150026E036A0250D76E0050FE
:10223000D66EE4CF03F0E4CF02F0E4CF01F0E4CFB8
:1022400000F0E4CFD9FF1200D9CFE5FFE1CFD9FFED
:1022500000C0E5FF01C0E5FF020EDBCF00F0030E7A
:10226000DBCF01F00050010A02E1015001E008D08B
:1022700061EC12F0006E005002E0E86A01D0010E3D
:10228000E4CF01F0E4CF00F0E4CFD9FF1200D9CFC2
:10229000E5FFE1CFD9FF00C0E5FF01C0E5FF020E79
:1022A000DBCF00F0030EDBCF01F00050010A02E1AA
:1022B000015001E006D09E9ABBEC11F0006E005078
:1022C00001D0020EE4CF01F0E4CF00F0E4CFD9FF5B
:1022D0001200D9CFE5FFE1CFD9FF00C0E5FF01C073
:1022E000E5FF020EDBCF00F0030EDBCF01F0005064
:1022F000010A02E1015001E005D09EAA02D0010EC0
:1023000001D0E86AE4CF01F0E4CF00F0E4CFD9FFD8
:102310001200D9CFE5FFE1CFD9FF00C0E5FF01C032
:10232000E5FF020EDBCF00F01F0E6F1600506F129C
:10233000E00E6F14016E01500018FAE1E4CF01F0D5
:10234000E4CF00F0E4CFD9FF1200E8AE06D0F3CF1F
:10235000EAFFEE50EECFF3FF1200E8BC0BD0E9CF5E
:10236000F6FFF3CFF7FFF86E0900F5500900F5CF3F
:10237000F3FF12001200F00E0001C215C26FABACE9
:1023800004D0C291ABA001D0C281ABA402D00001A5
:10239000C285ABA202D00001C287AE501200D9CFD5
:1023A000E5FFE1CFD9FF580EE56E000EE56E010E98
:1023B000E56ED6EC10F0030EE126E4CFD9FF120053
:1023C000E8AE04D0F3CFEAFFEE501200E8BC08D02C
:1023D000E9CFF6FFF3CFF7FFF86E0900F5501200D2
:1023E0001200D9CFE5FFE1CFD9FF020EDBCFA9FF65
:1023F000A69CA69EA680A850E4CFD9FF1200D9CFF4
:10240000E5FFE1CFD9FFD08EF28AF184F28EF36A34
:10241000010EE4CFD9FF120017EEFFF027EEFFF018
:10242000F86AA68EA69C9BEC0EF02DEC09F0FFD767
:10243000E8AE07D0F3CFEAFFE4CFEEFFF4CFEEFF34
:102440001200E8AC12001200E8AE05D0F3CFEAFFAC
:10245000E4CFEEFF1200E8AC12001200617B0080B6
:10246000AA0080000001020304050000ACAC04D007
:10247000AC900001C2B3AC80AD6E1200D9CFE5FFC5
:10248000E1CFD9FFE4CFD9FF1200D9CFE5FFE1CFEB
:10249000D9FFE4CFD9FF1200D9CFE5FFE1CFD9FFB3
:1024A000E4CFD9FF1200D9CFE5FFE1CFD9FFE4CFC8
:1024B000D9FF120001005C2400007B0000000F0027
:0A24C0000000000EACA2010F120094
:020000040030CA
:0E000000FFF2FFFEFFFFBBFFFFFFFFFFFFFF52
:00000001FF
